:020000020000FC
:1000000072CDA3C1000000001FC000008CC0000022
:10001000000096C00000000000000000020304067B
:10002000080C10182030406080000406080C1018DE
:100030002030406080A0C0000003070F1F000505AE
:100040000D050305030302004FB662FD0CC05520E9
:1000500041F00994C52DC095089483FDC795C4BD92
:1000600064604FBE1895C0916400089483FDC795E5
:10007000C4BD6B7FC0916400CF3F09F41DC070FF09
:1000800019C082FD05C04FBEC098C198C29818958E
:10009000C098C198C29876FD0DC064FD0BC0C9E040
:1000A000CA95F1F7C091B100C0FD939AC1FD949A31
:1000B000C2FD959A4FBE189524BCCC27C064C8BF1A
:1000C0006460F8CFC7CF70FFC5CF64FDC3CFC09ABF
:1000D000C1CF70FFBFCF64FDBDCFC19ABBCF70FF52
:1000E000B9CF64FDB7CFC29AB5CF939870FFB2CFA6
:1000F00064FDB0CFC7E0CA95F1F7C09AABCF949832
:1001000070FFA8CF64FDA6CFC7E0CA95F1F7C19AEA
:10011000A1CF959870FF9ECF64FD9CCFC7E0CA9594
:10012000F1F7C29A97CF4FB6C9B7CF7EC9BF6E7FDE
:10013000CCB5CE0DDDB5DF1DDBBDCABD4FBE1895FC
:100140003FB68F7EABB7A074A2118061A0E0ABBFB9
:10015000A9B7AE7FA9BF7894A0916800AA2341F007
:1001600085FD2EC0A0916800AA95A093680028C0C4
:1001700040E050E085FD14C0A0B396FDA095A2FD1F
:100180004FEFA3E096FDA2E0A5BFAA27A064AABFF7
:100190008D7FA0B396FDA095A2FD5FEF451741F7B7
:1001A000A8E161FDA093680085FD03C0A8E1A093CC
:1001B0006800409396008160442311F020929900DA
:1001C00085FD0EC0A0916900AA2331F0A0916900BD
:1001D000AA95A093690004C08061AA27A064AABF61
:1001E00080FF3DC0A09196004A2F61FF8E7F85FD64
:1001F00018C0403F08F040EFA42FA295AF704A0FFF
:100200005091B600533069F0A695A69550FD01C0F7
:10021000A69552FD03C0A41B4A2F03C04A0F08F441
:100220004FEFA0919F004A1708F44A2F40936100B6
:10023000A72FA670A1F073FD12C0A0917000AA0FA5
:10024000AA0F50919E0056955695541708F0452FC9
:100250004A0F4093610018F4AFEFA0936100A091A2
:100260006100A093630040916300A0919B004A1736
:1002700008F04A2F542EA091A000AA2309F422C00E
:10028000542F5A1B10F4A42F50E0BA2E8894AA1FA2
:10029000AA2EA091A200A095AA22A50E58F0A09186
:1002A000A100A21509F0AA95AA0EA093A10048F0FA
:1002B0004A2D08C0A091A100BA1608F0A395A093FA
:1002C000A1004FEF409364007F7B485F08F07064AB
:1002D000A0916000A395A093600051F0F894A9B795
:1002E000A160A9BF84FF02C0A0E4ABBF3FBE1895C8
:1002F000A0917400A395A093740041E05091680010
:10030000552329F085FF03C05A9550936800A091AA
:100310009600A13018F0209299000DC020929A000A
:100320002092A300A0919900AF5FA093990018F0CC
:10033000AFEFA0939900F894A9B7A160A9BF84FF7B
:1003400002C0A0E4ABBF3FBE18953FB64CB55DB54B
:100350008F7EABB7A074A2118061A0E0ABBFA9B73C
:10036000AE7FA9BF789481FD23C0A2E096FDA3E0F3
:10037000A5BF8260A0B396FDA095A2FF05C04093E3
:100380006500509366003EC1A3E096FDA2E0A5BFC4
:10039000AA27A064AABF8D7F85FF01C026C140E0C7
:1003A000A0B396FDA095A2FD20C1409396000FC179
:1003B000A3E096FDA2E0A5BF8D7F61FF71C0A2E022
:1003C00096FDA3E0A5BFAA27A064AABF82604093C0
:1003D000910050939200A0908F004A19B090900025
:1003E0005B09BB24A22C4C38520518F420929500CE
:1003F00049C0A091D400AA2359F1483C520528F4E1
:10040000A0E1BA2EAAE0AA2E23C04836A1E05A07DE
:1004100028F4A8E0BA2EAFE0AA2E1AC0403DA2E010
:100420005A0728F4A4E0BA2EAEE1AA2E11C0403A31
:10043000A5E05A0728F4A2E0BA2EACE3AA2E08C021
:100440004839A8E05A0720F4A1E0BA2EA8E7AA2E5E
:10045000C42EA0919300CA1AD52EA0919400DA0A56
:10046000DD202AF4AFEFC094D094CA1ADA0A2092A1
:100470009500A8E0A210A0E0CA14DA0618F4A1E0E2
:10048000A093950040939300509394004091910065
:100490005091920040938F005093900042E097C09B
:1004A000A09165004A1BA09166005A0B94FD82C082
:1004B00093FD80C092FD7CC086FF03C0D52EC42E64
:1004C0000CC05695479591FD73C05695479590FD84
:1004D0006FC0D52EC42ED694C79461FD19C0AC2D23
:1004E000AC51AD2DA24008F005C0DD2089F4AC2D43
:1004F000A85C70F4A0916700A395AA2311F0A093C3
:100500006700AA3008F471C02092960081606DC027
:10051000A0916700AA2319F0AA95A0936700A22CC6
:100520005091BA0097FD06C0A090C800533011F456
:10053000A090D000AAEFAA0EA22DA21DCA18DA0A16
:100540004FB74170533049F4442321F087FD05C073
:10055000806803C087FF01C08F77442359F0533070
:1005600031F4AFEFC094D094CA1ADA0A03C040E065
:1005700050E020C0533049F4CC0CDD1CAAE0CA1A6C
:10058000D20818F4A0E0CA2ED22CAFEFCA16D204BB
:1005900018F04FEF50E00EC0A091AC00CA9E412D64
:1005A000000C441F50E008F012C04FEF50E00FC0A5
:1005B0005695479594FF07C0552309F04FEFA42F98
:1005C000A6954A0F521D4F3F520508F04FEF40933A
:1005D0009600816061FF09C0AFE1A095A923AB2916
:1005E0009A2F8F7DBB2009F48062A8E1A093680058
:1005F00085FF03C0AAE0A093680061FD03C085FDEC
:1006000001C08F7E85FD03C0A6E0A0936900F89429
:10061000A9B7A160A9BF84FF02C0A0E4ABBF3FBEE1
:10062000189511E00AC013E008C01AE006C01EE1E8
:1006300004C014E602C018EC00C005E1BB27BA955F
:10064000F1F70A95D9F71A95C1F708952AE338E723
:1006500009C020E33CE806C02AE234EB03C025E2EF
:1006600038EC00C0B091AD00BA9509F4089512E0DD
:10067000BB279498BA95F1F7C19ABA95F1F7C1984A
:10068000BA95F1F7949ABA95F1F7123009F0C09A39
:10069000123009F4C29AB091AD00BA95F1F7123058
:1006A00009F0C098123009F4C298B7E8BA95F1F78A
:1006B0001A95F1F6022FB22FBA95F1F70A95D9F7EC
:1006C0003A9581F694980895221B39E0001F3A95D7
:1006D00009F40895221F211B18F4210F8894F6CFE6
:1006E0000894F4CF622C722CB0E08894B395221F4A
:1006F000331FE0F7379527958894912E802E020BB3
:10070000130B10F4192D082D10F4889401C00894CF
:10071000661C771CBA9571F7172D062D0895322D9A
:1007200011232AF43A9500951095031B130BF894A6
:10073000029F712C002D129F912C802C7894780CA4
:10074000172D921C292DB4E06B2E26951795079531
:100750006A94D9F7332321F000951095031B130BEE
:100760000895089510917B00169500917A000795E1
:10077000B0917E00B01B0B2FB0917F00B10B1B2FEF
:1007800028F40038BFEF1B0740F009C00F371205EF
:1007900008F405C00FE710E002C000E81FEF009367
:1007A000830010938400089500918300B09180002D
:1007B0000B0F10918400B09181001B1F20E030913D
:1007C000840033230AF42A95B09182002B1F1AF477
:1007D000203F40F00AC02F3008F407C00FEF1FEF92
:1007E0002FE003C000E010E020EF30916300B091F3
:1007F0009B003B1718F4323030F009C0B0918400F0
:10080000BB235AF004C0B0918400BB2332F40093A0
:100810008000109381002093820008952091D700DA
:1008200000918300000F10918400111F78DF1123C5
:100830002AF40038BFEF1B0740F009C00F3712053C
:1008400008F405C00FE710E002C000E81FEF002326
:1008500052F0B0916200B01B0B2F18F0013008F07D
:100860000AC001E008C000950F5FB09162000B0F55
:1008700008F001C00FEF0093850008952091D80083
:1008800000918100109182004ADF11232AF4013087
:10089000BFEF1B0740F009C00F3F120508F405C069
:1008A0000FEF10E002C001E01FEF112352F0B091F2
:1008B0008500B01B0B2F18F0013008F00AC001E0D2
:1008C00008C000950F5FB09185000B0F08F001C0C4
:1008D0000FEF0093630008950FEF71FD1EC0B091FC
:1008E000D300BB23D1F0B0917B00BB23B1F00FEF5D
:1008F00010917B00E9DEF894B091730072FDB5E0D1
:100900000B9F112D002D7894112309F00FEFB0915A
:100910009E000B1710F400919E0000939D00089517
:1009200000917A0010917B0000541140B0919D001D
:1009300010F4BA9501C0B39511F0B0939D000895DD
:1009400000C008952091B500B6B1B6FDFBCF04B14B
:1009500015B1B6B1BF77B6B9B091AA00B395B0934F
:10096000AA00B83060F12092AA00B091D200BB2357
:1009700021F1112329F0B091AB00BF3F61F009C014
:10098000B091AB000B1739F020F4BB2321F0BA95DE
:1009900002C0B395E1F300919B00B093AB00BA3F66
:1009A00050F400ECB93F38F400E8B83F20F400E41C
:1009B000B73F08F400E000939B007F7E0895B0915C
:1009C0009B00B39511F0B0939B00B091AA00B73093
:1009D00009F47061089502E3F894B091D9000B9F77
:1009E000012D000C001F7894B0919B000B1710F0A4
:1009F00000919B000093610000936300502E0093D0
:100A0000640000939E00089520927A00B0EFB093A6
:100A10007B000895F8940CB51DB52091740078946E
:100A20003091750060907600009375001093760009
:100A3000031B160971FD03C077FD80C028C07090AC
:100A40007700209377002709222319F00FEF1FEF7B
:100A50000EC080907800909079003093780060927A
:100A600079000091750010917600081919092091FC
:100A70007A0030917B0036952795020F131F10F4F2
:100A80000FEF1FEF00937A0010937B002BC0209193
:100A90007A0030917B003901B4E08B2EB2E09B2EBE
:100AA000343040F08A949A94383020F072FD02C0BD
:100AB0008A949A94769467948A94E1F72619370970
:100AC000992021F0169507959A94E1F7200F311F90
:100AD00020937A0030937B0028F43FEF30937A0024
:100AE00030937B00323008F4706871FF02C0B3E0CD
:100AF0000DC0B091C40000917100023838F0B39578
:100B0000003A08F0B395B63008F0B5E09B2EB4E09B
:100B10008B2E10917B0000917A0024E016950795AA
:100B20002A95E1F70819120928F0B02FB250B12F19
:100B3000B20910F402E010E0980126C020917A007A
:100B400030917B003901769467946694669466943C
:100B50002619320906950695200F321D20937A003A
:100B600030937B00323008F07F7704E0369527958C
:100B70003695279526952695201B10F0223008F4EF
:100B800022E089019090C40060FDFECFE0908B00D0
:100B9000F0908C006160B9B7B061B9BF380177FDE2
:100BA00041C07694679400938B0010938C00B92D0C
:100BB000B330E1F0B0FD04C0060D171D930106C06F
:100BC000000F111F0250120922E030E0B92DB3309E
:100BD00068F020938D0030938E000093870010936F
:100BE00088006092890070928A003AC000938D005C
:100BF00010938E00209387003093880060928900C4
:100C000070928A0071FF0DC0BFE0B0938D002092FA
:100C10008E00B093890020928A00B0938B002092BE
:100C20008C001EC0669400938B00B92DB33091F0F8
:100C3000B0FD03C0060D262D03C0000F025022E0B8
:100C4000B92DB33038F020938D0000938700609267
:100C5000890006C000938D00209387006092890070
:100C600000917C0002FD0350013031F495FD0FC06E
:100C7000B0B7B77FB0BF11C0023039F4B0B7B860B9
:100C8000B0BFB4E0B06CB7B908C095FDF1CFB0B754
:100C9000B860B0BFB5E0B06CB7B90091A200000F6A
:100CA00010F4BBE60B270093A20060FDFECFB2E07C
:100CB000B0936E006160B9B7B061B9BFB72FB670BD
:100CC000D1F020917A0030917B00369527953695AA
:100CD000279571FF02C0B0E43B0FF8940CB51DB529
:100CE000020F131F1BBD0ABD6160B0E1B8BFB9B7E9
:100CF000B061B9BF78940895686020927D0020E0CB
:100D000066FD20E206C0686020927D0020E266FD5C
:100D100020E001E011E077FD11C0B72FB67009F0B7
:100D2000677F14E100917B00069509F403950F306D
:100D300008F00FE071FF02C004E114E160FD0FC094
:100D4000B0917D00BB2359F071FF06C0B0916E00D9
:100D5000BA95B0936E0011F4706251C0ABDFB0B7BA
:100D60003B2FB77FB0BFB8B1B0B733FDB860B0BFED
:100D7000B0917D00B395B0937D00B8B177FD06C00A
:100D8000B1E071FDB3E0BA95F1F7B8B1B072B21746
:100D900009F02AC071FF05C00395011708F00A95F4
:100DA000CDCF63FD05C00395011708F0B2CFC6CFC4
:100DB000677FF8943CB56DB470907A00B0917B0079
:100DC000770CBB1F08F4BFEF770CBB1F08F4BFEF15
:100DD000370D6B1E6BBC3ABD6160B0E1B8BFB9B7EF
:100DE000B061B9BF789495CFB0916D00B13008F47F
:100DF00090CF63FD8ECF0A9509F0A0CF7F7D209123
:100E00008D0030918E00F894B0E1B8BF0CB51DB5DF
:100E1000020F131F1BBD0ABDE0908700F0908800F1
:100E20006160B9B7B061B9BF7894B72FB67039F0C7
:100E3000B0916D0072FFB395B0936D0009C075FF5E
:100E400007C066FD05C063FD03C0BF91BF91FFC42D
:100E5000089500E063FF01C001E0F8941091710073
:100E6000B7E01B9F212D102D7894200F2695179504
:100E7000269517952695179510937100183718F435
:100E8000B8E7B093710000917100B09172000B1738
:100E900020F06061C098C198C29860FDFECFE090DC
:100EA0008900F0908A006160B9B7B061B9BF089558
:100EB000B2E095FD0AC0F894B0937C009498939AA0
:100EC00062FF01C0C29A7894F4C0F894B0937C0099
:100ED0009498959A62FF01C0C09A7894EAC0B3E0F2
:100EE00082FF24C095FD11C002E0F894B0937C000D
:100EF000EFE7F0E00093B100C298959862FF02C05E
:100F0000C19A01C0949A7894D4C002E0F894B09346
:100F10007C00EFE7F0E00093B100C098939862FF87
:100F200002C0C19A01C0949A7894C3C095FD0BC0C9
:100F3000F894B0937C00E9E6F0E0C29862FF01C04B
:100F4000C19A7894B6C0F894B0937C00E9E6F0E0DA
:100F5000C09862FF01C0C19A7894ABC0B4E095FD1F
:100F60000AC0F894B0937C009398959A62FF01C0F0
:100F7000C19A78949EC0F894B0937C009598939A07
:100F800062FF01C0C19A789494C0B5E082FF24C08A
:100F900095FD11C001E0F894B0937C00E5E7F0E026
:100FA0000093B100C198949862FF02C0C09A01C03A
:100FB000939A78947EC004E0F894B0937C00E9E8BA
:100FC000F0E00093B100C198949862FF02C0C29A09
:100FD00001C0959A78946DC095FD0BC0F894B093BC
:100FE0007C00E3E6F0E0C19862FF01C0C09A78940B
:100FF00060C0F894B0937C00EFE6F0E0C19862FF27
:1010000001C0C29A789455C0B6E095FD0AC0F89424
:10101000B0937C009598949A62FF01C0C09A78942E
:1010200048C0F894B0937C009398949A62FF01C0F2
:10103000C29A78943EC0B1E082FF24C095FD11C0F1
:1010400004E0F894B0937C00E9E8F0E00093B1008C
:10105000C098939862FF02C0C29A01C0959A789492
:1010600028C001E0F894B0937C00E5E7F0E000933D
:10107000B100C298959862FF02C0C09A01C0939ACD
:10108000789417C095FD0BC0F894B0937C00EFE600
:10109000F0E0C09862FF01C0C29A78940AC0F89448
:1010A000B0937C00E3E6F0E0C29862FF01C0C09A12
:1010B00078946F7E089522E630E0F9012092B10025
:1010C000C098C198C2989398949895986B7F08950A
:1010D000A2EBB0E00FEF0D930D930D930D9303E092
:1010E0000D9304E00D9309E00D9303E00D9301E0EF
:1010F0000D9301E00D93AEEBB0E001E00D930FEF27
:101100000D930D930D930D930D9303E00D930FEF3E
:101110000D930FEF0D930D9305E20D9300ED0D93DD
:101120000AEF0D930AEF0D9304E00D930FEF0D936B
:1011300001E00D9300E00D930AE70D930FEF0D937F
:1011400000E00D9301E00D9300E00D9303E00D939B
:1011500000E00D9308952091B9008B7F233009F4AE
:101160008460B091BA00B33019F09F7DB1FD9062F8
:101170009F7BB091BB00B1FD9064223011F088607C
:1011800001C0877F08950A95E00FF21DB49108957C
:10119000ECE1F0E00091B200F6DFB093D700ECE1B3
:1011A000F0E00091B300EFDFB093D800EAE2F0E0A6
:1011B0000091B800E8DFB093D9000091B800023088
:1011C00008F402E000937300B091CE000FEFB2304C
:1011D00009F400EAB33009F402E800937200E8E38E
:1011E000F0E00091D500CFDFB093A00008950895FE
:1011F0002091C8003091C900B091BA00B33009F411
:101200003E5097FF02C020E03FEFB32FB21B6B2E82
:10121000B25810F4B2E86B2E00E00395609EB12D39
:10122000BD57D8F30093AC0008959068E1DFFFD973
:10123000FED920E030E0B0E16B2EF5D9B0919600F8
:101240002B0F321D6A94C9F7B4E036952795BA95ED
:10125000E1F7822E9F77CCDF0895F894E3E0F0E089
:10126000B9E0B7BFB491B078C1F3F894A895B1B51F
:10127000B861B1BDB0E0B1BDB4E0BEBFBFE5BDBFB8
:101280001ADFB0E0B8BBB7E1B7BBB0E0B5BBB0E0C8
:10129000B4BBB0E0B2BBB8E3B1BB2224A0E0B0E085
:1012A0002D92AA31E9F7A0E6B0E00FEF2D920A9552
:1012B000E9F7B1E0B093A2000BDF05D3B0E0B06C6A
:1012C000B7B9B6B1B460B068B6B90091CA000093BE
:1012D000AD00B1E0B0936A00F894ADD9B7D9A7D901
:1012E000B8D9A5D9B9D9A3D975D3A5D9A4D9A1D924
:1012F000F8940AEF1AEFA0B396FDA095A2FF1FC0C5
:101300001A95C9F70A95B1F7E0E0FCE1B591B43E52
:1013100039F4B591B03E21F4B591BF3F09F40CC04A
:10132000E0E0F395F395B591B83F49F4B591B43940
:1013300031F4B591BA3A19F4EE27F69509940BDF1A
:1013400027DF55DF55DF0091CA000093AD00B3DE03
:10135000B2E0B3BFB2E0BEBDB2E0B5BDB1E5B8BF6B
:10136000B9BFB0B70B2FB77FB0BFB8B1B0B703FDEF
:10137000B860B0BF56D97894E3DA20927000B3E039
:1013800096FDB2E0B5BFB0E4BBBFBB27B064BABF47
:101390008D7F51D9626033E02CE0B0919500BB2382
:1013A00021F42CE03A9509F4A3CF41D980FFA0CFD6
:1013B0008E7FB0919600B23078F3B92FBF71009153
:1013C000980000939700B0939800B01729F72A95DA
:1013D00021F76D7FB3E096FDB2E0B5BFBB27B064E7
:1013E000BABF8D7FB091D400BB2321F48062B92FA6
:1013F000B0709B2F8F7B209267001BD985FF05C0A3
:10140000B0916700BA3008F080640DD902E085FF22
:1014100001C000E0B0919600B017B8F3F89416D967
:1014200015D914D9789407D920928600B091BA00C2
:10143000B33009F47EC0F7D8B091BE00B13008F4E3
:1014400078C0B0916A00B13008F473C085FD18C04F
:10145000B0919600BF3F08F46CC0F89400D978941E
:10146000E8D8B0919600B130C0F7F894EFD8DDD845
:10147000EDD87894DED8B0919600BF3FB0F3DCC2CF
:10148000B8E09B2E9068F894B3DE7894D2D8F894A4
:101490009F77AEDE80909600B0919600BF3778942B
:1014A00008F44FC0BED8F894DAD878949A9451F7DB
:1014B000BCDEB82DB550B093C900BDD8F8948FD21A
:1014C0007894BAE09B2E9068F89492DE7894B1D824
:1014D000F8949F778DDE80909600B0919600BF378C
:1014E000789478F79ED8F894B1D89FD8AFD87894EC
:1014F0009A9449F79ADEB82DBB5FB093C8000B2FC2
:101500001091C900125810F0100B20F4B2E80B0F24
:101510000093C90090D8F89403D270D2789489D8F7
:10152000F89466DE7894B0919600BF3F08F48ECFB1
:1015300083C200919600B09186000B1710F00093C3
:10154000860077D801E0B091BA00B35009F405E005
:10155000B0919600B01708F069CFF89480D87FD882
:101560007ED8789468D820926A0020926B002092EE
:101570006C00B0916B00B395B0936B00BF3F71F5F9
:10158000B0916C00B395B0936C00B091CC0009E1C0
:10159000BA9559F002E3BA9541F00DE7BA9529F0F2
:1015A0000AEFBA9511F020926C00B0916C00B01760
:1015B000A8F081DD36D8B0916C00BA95B0936C007C
:1015C00020926B00B091CB00B093AD00F89447D857
:1015D0007894B091CA00B093AD002BD826D8B091C2
:1015E0006800BB2319F485FF01C082CE01E085FDB0
:1015F00001C006E0B0919600B01708F4BACFB091E0
:10160000BA00B35009F015D8B0916800BB2309F4B3
:101610006FCEF89450DD20926100209262002092FB
:101620006300522C209264002092A1007894B09123
:10163000B700BB0FB0939F0020927E0020927F00E6
:101640002092800020928100209282002092AA00A5
:1016500060E070E020927100B8E0B093AA00706181
:10166000E0D7B0E074FDB1E0B06CB7B9B6B1B06826
:10167000B064B6B9B6B1B6FDFDCF04B115B1B6B11F
:10168000BF77B6B9112309F00FEF0093AB005AD919
:10169000B8E0B093AA0070615EDDF894BFEFB0933C
:1016A0009B0099D9B0916100B0939B00B0939C00CE
:1016B000B0939D007894B1E0B0936100B093630063
:1016C0005B2EB0936400B093A400B0919A00B093E5
:1016D000A300B091BA00B33019F49F7D87FD9062EA
:1016E0007160726020926D008FDCA5DC8DD992D97B
:1016F0008BD990D989D907DB34D8ABDBD9DB8AD930
:10170000FBDA65FD2FD877FFE7D877FD09D9A1DB94
:10171000E6DB80D9F8DA65FD47D89BDB1FDC7AD998
:10172000EBDA65FD7BD895DB30DC74D9ECDA65FD4E
:10173000A5D88FDB69DC6ED9DFDAB0E074FDB1E0EB
:10174000B06CB7B9B6B1B068B064B6B982DB73DC5F
:1017500061D9F8D871FF21C0B0919E00B0939B0071
:10176000B0939C00B0919A00B093A300B1E0B09305
:10177000A40018E12CE0B0916D00B11740F07D7F1E
:10178000746020936F00BFEFB0939B0006C0B091D0
:101790009600B13008F0AFCF64C072FF15C066FD8F
:1017A00013C0B0916F00BA9519F47B7F7860A3CF16
:1017B000B0936F00B0919600B13008F09CCFB0911B
:1017C000BA00B33009F04DC020927000B09199007A
:1017D00002E81091D600112309F003E0B01708F0D9
:1017E00040C085FF04C0B0916800BB23D1F1B09127
:1017F000BA00B33081F495FD03C087FD04C00BC06F
:1018000087FF01C008C066FD06C06064B0919E00FD
:10181000B0939B0085CF00EF66FF05C0B0919E009E
:10182000B0939B0000E2B0917B00B01708F463CF47
:1018300066FF17C06F7B9F7D87FD90627460B2E189
:10184000B0936F00B0919E00B0939B0054CFB091C5
:101850007000B395B0937000B0919600BB2309F06F
:1018600002C020927000F89426DC8090B900B2E0AB
:10187000B093B90070DC8092B90020926100209290
:10188000620020926300522C2092640020929F00FC
:1018900060E070E07894CDD60EDC0091D600002395
:1018A00019F0C09AC19AC29AB0E0B06CB7B9B6B19B
:1018B000B460B068B6B985FF05C0B0917000B430AF
:1018C00008F016CD52CEEDE0F0E023D00A3509F055
:1018D0001BC0EEE0F0E01DD0053A09F015C03AE07B
:1018E000A2EBB0E0E3E0F0E014D00D9331963A952E
:1018F000D9F739E1AEEBB0E0EFE0F0E00AD00D93BC
:1019000031963A95D9F702C0E3DB0AD0E8E2F0E07D
:101910000895E199FECFEEBBFFBBE09A0DB30895A9
:101920001ED03AE0A2EBB0E0E3E0F0E00D910FD082
:1019300031963A95D9F739E1AEEBB0E0EFE0F0E05F
:101940000D9105D031963A95D9F712D00895E199C5
:10195000FECF0DBBEEBBFFBBE29AE19A0895EDE02E
:10196000F0E00FEFF4DFEEE0F0E00FEFF0DF0895CE
:10197000EDE0F0E00AE5EBDFEEE0F0E005EAE7DFBE
:1019800008953091AE000091AF00313011F4009312
:10199000B600323011F40093B700333011F40093E5
:1019A000B800343011F40093C400353011F40093C2
:1019B000B900363011F40093D500373011F400939C
:1019C000CE00383011F40093BA00393011F400938E
:1019D000BB00089525E02FD62A95E9F7089536D65D
:1019E00038D63AD63CD621D631D633D635D637D6A8
:1019F0001CD62CD62ED630D632D6089530D62CD63C
:101A000028D624D612D62BD627D623D61FD60DD627
:101A100026D622D61ED61AD608958090AE00909073
:101A2000AF0014D613D612D600D68A94D1F717D6A3
:101A3000FCD59A94E1F70895F894D1DF7894CADF41
:101A4000C9DFB1E0B093AE00B1E0B093AF00209237
:101A5000B000F894E2DF7894B5E06B2E70909600B9
:101A6000EAD5B09196007B16C9F7B13018F0BF3FA8
:101A700040F107C086DFF89453DFB1DFB8E0B1BDB5
:101A8000A9DF6A9459F7B091B000B395B093B00054
:101A9000B33008F4DECF9EDFB091AF00B395B093C2
:101AA000AF00F894B091AE00BA95EEE3F0E0EB0F22
:101AB000F21D049178940395B091AF00B01708F42B
:101AC000C6CF88DF87DFB091AE00B395B093AE008C
:101AD000B091AE00BA3008F4B7CFFADAF89420DF4C
:081AE000B8E0B1BD77DFB9CB1E
:00000001FF
